:020000040000FA
:020000001628C0
:08000800312C82073F3406345D
:100010005B344F3466346D347D3407347F346F3451
:1000200000340234043408341034203403138312AF
:100030008501860187019F018316031788018901C5
:10004000031375308F00F030850001308600870182
:10005000C3308100831200308B00860186170000B8
:100060003230051B3C30A100A3000310A30CA30CED
:100070000B168B178030A20086018614221C871471
:10008000221807142C248701860106170000051F7B
:100090003C288601A2012108A3001230A500A60178
:1000A000A7010130A400AC00AE01B101B001B40160
:1000B000B201B601B7018316A73084003C30A4001A
:1000C0008001840AA40B6028831234170630810053
:1000D000FA30A0008B1631187828AD01AB01240846
:1000E00081222508A9002608AA00B71BB71DD22225
:1000F000C030B405023086002B0887002C24E22093
:1001000000308700043086002A080F390520B71F09
:100110008B28371A803887002C24E2200030870093
:10012000083086002A0E0F390520B71F9928371A84
:10013000803887002C24E2200030870010308600B1
:1001400029080F39052087002C24E2200030870081
:1001500020308600290E0F39031DB128B71BB71DAB
:100160000A30052087002C24E22000308700403030
:1001700086002C0887002C24E22000308700803085
:1001800086002D0887002C24E2200030870086019D
:100190003408C0390319DF28341BD0280F21DF2889
:1001A000B41BDF2834081F39153C031DDF28200845
:1001B000031DDF28063081004B30A0008B1630185D
:1001C00092236B28B41B0E290508F039B300B31B2A
:1001D000B713B31FB717331A06290730B407B31A7A
:1001E00006290730B407331BFF281F303405143CA1
:1001F0000319FD280D30B4020E29B40A0E291F3050
:100200003405143C031D0629B71FFD28341B0E2995
:10021000B417063081001930A0008B16080034088E
:100220001F39B5003618172931181B293114A82297
:10023000AF01B801B6010A30350203184C29AF1FCF
:100240002829A822AF13311D2829310E0339AB000C
:100250000430B9000310AA0DA90DB90B2A293508DD
:10026000AA042908F03903193929A03C031D4B2998
:100270003B29A030A90429080F39031943290A3C56
:10028000031D4B2945290A30A9042A08F039031D0A
:100290004B29A030AA046D2A0C30350203185C29C2
:1002A000AF1BA822AB01351CAB1435182B140F3033
:1002B000B1052B0EB1046D2A0E30350203189929B1
:1002C0003808031D88292A080F39BA000A3C031987
:1002D0008F293518782908303A02031898293A08E6
:1002E0008122E330AF05BA0D3A0D1C39AF048529E0
:1002F000AC0105303A02031898293A089122E030FF
:10030000AF053A080339AF04B114B817AB229829E6
:10031000B81E8D298030B8059229381B92293223C6
:1003200038179829A822351C7C2235188F223813BB
:100330006D2A113035020318FE29B11C662A351AC0
:10034000AA29351CAB1635182B179F30AF05351C65
:10035000AF16AD29AB176030AF042B080339031972
:10036000B9292C08031DEE29311D662A8F227C2213
:10037000EE292C08031D662A2A080F390A3C0319A6
:10038000C3298F22E1292D080319662A351AD0299D
:100390002D08351C8504FF3A351885053110FD29D7
:1003A0000130A900AA010023AF12A9177323031873
:1003B000642AA913D2227C22AB132B172D088504A3
:1003C000FD293214AF220318662A0023A9177323CC
:1003D0000318642AA913D2227C22FD293210AF22ED
:1003E0000318662A0319C3292908BA00ED227323CA
:1003F0000318642A3A08A90031156D2A031D052A3D
:10040000B1103111AF01A8226D2A13303502031843
:10041000412A0330AD08031D112A1C30AC08031912
:10042000292A8316A60083122F088316A000A7305E
:1004300084001430A400801F232A2008260500060B
:1004400026050319800103308407A40B1B2A83129D
:100450003F2AB71F332AB70A37080739053C031D5F
:10046000402AF830B7058316A73084003C30A4003A
:100470008001840AA40B382A8312B71F8501B101B9
:100480005D2A031D602AAF1B5D2A2C0803195D2A13
:100490002B08033903195D2AB201AF220318662A1B
:1004A00003195D2AAF0C2F0C073903190130A40082
:1004B000ED222908A5002A08A600AC01B1016D2A89
:1004C0000830B70631106D2A8830672A9930AA00A3
:1004D000A900AB01AC01AD0136140C303502031993
:1004E000752A0D303502031DB80112303502F8307F
:1004F000031DB705341708002F08B900B90C390CD3
:10050000073903198C2AB9000130AC00B90303196B
:100510008E2A0310AC0D862A7F30AC0008002F080D
:10052000033903190430B9000130AD00B9030319D0
:100530009C2A0310AD0D962A08000330AB0540300D
:10054000AF1EA62A20302F1FA62A8030AB04080039
:10055000AB01AC01AD01AA30AA00A900080029082E
:10056000F039A03C031DBE2A0F30A90529080A3C1A
:10057000031DBE2A123032180030A9001330321881
:10058000123029020318D12A2A08F039A03C031D91
:10059000CF2A0F30AA052A080A3C0319D12A603055
:1005A0002A0208002908031DD82A1230A900DC2AD3
:1005B000123029020318DE2AAB14EC2A0319EB2AA5
:1005C000A9000E302902031CEB2A1030290203185F
:1005D000EB2A0630A9022B1408002908123C031943
:1005E000A9012B1CFF2A1230A9071A302902031C6B
:1005F000FF2A223029020318FF2A0630A907080023
:10060000E330AF052408BA00BA0D3A0D1C39AF0427
:100610002608AA072A080F39093C0630031CAA0736
:100620002A08593C0318172B6030AA02A90A25088A
:10063000A90729080F39093C0630031CA907290816
:10064000233C0318312B2430A9022F081C39043E07
:100650001C3903192E2B0430A007312BE330AF05D2
:100660002F1508002F088316A000831238081F39A1
:100670008316A500831235088316A600A7308400D0
:100680001430A400801F542B200826184B2B1C3933
:1006900000061C394E2B033900060339031D542B69
:1006A000250803195C2BA50303308407A40B422BF8
:1006B0008312B816A822722B00088312AF0083168B
:1006C000840A000883127F39A9008316840A00086F
:1006D0008312AA00B80AAB01B71BB71DD2227C2235
:1006E0008F229D2208008316A73084001430A400B6
:1006F000801F802B03308407A40B782B0314902BCE
:100700008312AF172F0883168000840A83122908EA
:1007100083168000840A83122A088316800003103F
:100720008312080024088316A1008312250883166B
:10073000A200831226088316A3000310A10DA10DA9
:10074000A73084001430A400801F112C00081C392D
:100750000319AD2B2106031D112C0008A000840AEB
:1007600000087F392202031D122C840A000823028C
:10077000031D132C20088312BA000339B900031992
:1007800039150130AE00B9030319C92B0310AE0DA2
:10079000C32B2E08BA1A8504FF3ABA1E85058316A4
:1007A0008403801FDA2B201FD72BA01ADC2B840395
:1007B0008001112C201F122C840320308006840A13
:1007C000A01AF42B2224F9300002031D122C23302E
:1007D00080001C30A0050319122C0430A002031D58
:1007E0000C2C1C30A0000C2C0008A600801319242F
:1007F0002430000203188001A61B80177F300005FB
:10080000031D122C1C30A0050319122C0430A00764
:10081000A01E0C2C0430A0008403E3308005A0004F
:100820008004840A840A840AA40BA42B8312301047
:100830000800800A00080F390A3C031D0800063032
:100840008007080000080F390319282C80030800CE
:100850008003063080020800C830BB00BB0B2E2C82
:100860000800F200030E8301F0000A08F1008A017B
:100870008B183D2C0B19582C632C8B10A30B4A2C76
:100880002108A300A21F522C0310A30CA30C0130BB
:10089000A206632CA21B632C0310210C2302031D50
:1008A000632C532C6A24B71F632C1030B706632CBB
:1008B0000B1106308100A00B632C8B12B41F622C2D
:1008C000B413632C341371088A00700E8300F20E87
:1008D000720E090027308400192460302702031C9F
:1008E000902CA70130142630840019246030260291
:1008F000031C902CA60125308400192424302502E5
:10090000031C902CA501A40A08302402031C8A2C85
:100910000130A4003118902C0310AC0D0318AC0D5D
:020920000800CD
:02400E00E423A9
:02401000FF3F70
:1042000043006F0070007900720069006700680069
:1042100074002000280043002900200032003000F4
:104220003100390020006200790020004D002E008E
:10423000590061006D0061006D006F0074006F0037
:00000001FF
